:10000000C728910190009F1727308F0010301420CF
:1000100003308F00E83014208F01643014208F01EA
:100020000A30142010081F288E0011088D001008B7
:100030008C0090200C08031D9F139F1B0800303E6E
:100040009200220884000930930003102C20920CA7
:10005000930B262803142C2884139F1D3B2800088B
:1000600020041F1D20068000841700082004031CA4
:1000700020068000462800082004031C20061F19C3
:100080002006800084172009800546281F0D0639A8
:100090008C004F208D008C0A4F2000006928003012
:1000A0008A000C0882070134753403341534003497
:1000B0003C340C34D9348F018E00FF308E07031C82
:1000C0008F07031CC22803308D00DF3069205D28B4
:1000D0008D01E83E8C008D09FC30031C72288C07D2
:1000E00003186F288C0764008D0F6F280C18782870
:1000F0008C1C7C2800007C280800930192001C3096
:100100008E006F308F00AC200F3083168104831275
:10011000FF3063008C07031C8D0703188928C22851
:1001200091019001103092000D0D900D910D0E086F
:1001300090020F08031C0F0F91020318A6280E0847
:1001400090070F0803180F0F910703108C0D8D0DEA
:10015000920B94280C08C228103094008D018C0159
:10016000930C920C031CBA280E088C070F08031876
:100170000F0F8D078D0C8C0C910C900C940BB028EC
:100180001008C22883130313831264000800831627
:1001900085010F308600831201307D20C03086003B
:1001A00005305B200608A400F03086000F302405DF
:1001B000A5000530A2000430A00006309F00FE30EC
:1001C0002020013020202030202020302020250831
:0801D0000120CC286300EA289D
:02400E00FD3F74
:00000001FF
